:10000000020012539507539607E5A254CF4410F50A
:10001000A222787FE4F6D8FD75813502001E120019
:08002000031202B5D2AF80FE0D
:10003B0002003EC0E0C083C082C0D075D000C002B9
:10004B00C004C005C006C00730D854C2D8AFDAC34D
:10005B00EF9448748094804015E50F2517F517E54C
:10006B000E3516F5168517EAE516F5FA8031E5DA41
:10007B005411602B852921852A22AFFA7529008F0F
:10008B002AE52AFEADEA7C00E42DF52AEC3EF529A3
:10009B00C3E52A9522F517E5299521F516D20030EF
:1000AB00D954C2D9AFDBC3EF944874809480401508
:1000BB00E5112519F519E5103518F5188519EBE536
:1000CB0018F5FB8031E5DB5411602B852B23852C38
:1000DB0024AFFB752B008F2CE52CFEADEB7C00E4E5
:1000EB002DF52CEC3EF52BC3E52C9524F519E52BC2
:1000FB009523F518D20130DA54C2DAAFDCC3EF9492
:10010B0048748094804015E513251BF51BE51235CB
:10011B001AF51A851BECE51AF5FC8031E5DC541158
:10012B00602B852D25852E26AFFC752D008F2EE59A
:10013B002EFEADEC7C00E42DF52EEC3EF52DC3E54B
:10014B002E9526F51BE52D9525F51AD20230DB6190
:10015B00ADBA43BA80C2DB90FD54E0C394487480BF
:10016B0094804016E5152509F509E5143508F508C1
:10017B00A3E509F0E508A3F0803590FD54E0541198
:10018B00602D852F2785302890FD56E0752F00F5C3
:10019B0030FE90FD55E07A002400F530EA3EF52F55
:1001AB00C3E5309528F509E52F9527F508D2038D82
:1001BB00BA30DF02C2DFD007D006D005D004D002A0
:1001CB00D0D0D082D083D0E032AD07ED6404702163
:1001DB00C2DEF5F9F5E912033FFFE5D954F14FF50E
:1001EB00D9900004120358640160030202B4D2DEFA
:1001FB0022ED7027900001120358FFE5F2543F4F98
:10020B00F5F2900002120385F50F85F00EC2008502
:10021B000E16F5178517EAE516F5FAED640170274A
:10022B00900001120358FFE5F3543F4FF5F3900094
:10023B0002120385F51185F010C201851018F5190E
:10024B008519EBE518F5FBED6402702790000112A0
:10025B000358FFE5F4543F4FF5F490000212038569
:10026B00F51385F012C20285121AF51B851BECE5FE
:10027B001AF5FCED6403703143BA80900001120350
:10028B0058FF90FD57E0543F4FF09000021203854A
:10029B00F51585F014C203851408F50990FD55E595
:1002AB0009F0E508A3F053BA7F22E4F53274FFF5A9
:1002BB0033F5347B007A007931E4FF1201D4E4F595
:1002CB003275337F7534FFFB7A0079317F01120170
:1002DB00D4E4F53275333F7534FFFB7A0079317F07
:1002EB00021201D4E4F53275331F7534FFFB7A002B
:1002FB0079317F031201D47531087535017B007A92
:10030B000079317F041201D4E4FB7D4D7F0412038D
:10031B00BDE4FB7D4DFF1203BDE4FB7D4D7F011260
:10032B0003BDE4FB7D4D7F021203BDE4FB7D4D7FDE
:10033B00030203BDBB010689828A83E0225002E7D8
:10034B0022BBFE02E32289828A83E49322BB010C47
:10035B00E58229F582E5833AF583E0225006E9250B
:10036B0082F8E622BBFE06E92582F8E222E5822925
:10037B00F582E5833AF583E49322BB0110E58229EC
:10038B00F582E5833AF583E0F5F0A3E0225009E925
:10039B002582F886F008E622BBFE0AE92582F8E200
:1003AB00F5F008E222E5832AF583E993F5F0A3E95A
:1003BB009322EBF582758300D39403748094805061
:1003CB0030E582700553B77FC2BFE5826401458378
:1003DB00700553B77FD2BFE5826402458370054336
:1003EB00B780C2BFE58264034583700543B780D2F3
:1003FB00BFEF14601114601214601314601D2404F9
:10040B0070248DDA80208DDB801C8DDC801843BA44
:10041B008090FD54EDF053BA7F800BED5401FFE556
:09042B00D954FE4FF5D97F0022DF
:00000001FF
